:020000040000FA
:100000008E018F01900191019201013093009401C2
:100010008501860198018316860110308500043021
:1000200081008312051EDF284220852098080319CD
:100030001B28851598030B1D1B288B01B1200C086C
:10004000143A031D2528860185018C0B1B281428D2
:100050000F398207FC340234D134B134673496341A
:100060009E348034FF34F13400340F398207003479
:1000700001340134043400340234023405340034D1
:10008000063400347A308C008E0A0E08093C0318BE
:1000900008007B308C008E018F0A0F08053C031886
:1000A000080079308C008F01900A1008093C031871
:1000B00008007B308C009001910A1108053C031860
:1000C00008007C308C0091011308003C0318732851
:1000D000920A1208023C03187D287D308C00013002
:1000E000920093017D28920A1208093C03187D288A
:1000F0007D308C009201930A7D28120898009308A5
:10010000031984280A30980708009501940A1408F6
:10011000063C031C94011408013A03199D28033A74
:100120000319A228013A0319A528073A0319A82898
:100130000030860000308500080095151308031D67
:10014000AA28080015151208AA2895141108AA282B
:100150001514100897002820860017083520850000
:100160000800051A0800950803190800970A1708DF
:10017000093C031C97011708AA20D720051EBE289A
:10018000D720051EBE2814309600051EB628D7209D
:10019000960BC528170894018F018E0195199300BD
:1001A00015199200951891001518900014280C301C
:1001B0008C000B1DD9288B018C0BD92808009601C7
:1001C0001608AA20D720D720960A16080A3A031D37
:0401D000E028DF281C
:02400E00F13F80
:00000001FF
